:100000000C9482040C94B2040C94B2040C94B204C8
:100010000C94B2040C94B2040C94B2040C94B20488
:100020000C94B2040C94B2040C94B2040C94B20478
:100030000C94B2040C94B2040C94B2040C94B20468
:100040000C94B2040C94B2040C94B2040C94B20458
:100050000C94B2040C941C090C94B2040C94B204D9
:100060000C94B2040C94B2040C94B2040C94B20438
:100070000C94B2040C94B2040C94B2040C94B20428
:100080000C94B2040C94B2040C94B2040C94B20418
:100090000C94B2040C94B2040C94B2040C94B20408
:1000A0000C94B2040C94B2040C94B2040C94B204F8
:1000B0000C94B2040C94B2040C94B2040C94B204E8
:1000C0000C94B2040C94B2040C94B2040C94B204D8
:1000D0000C94B2040C94B2040C94B2040C94B204C8
:1000E0000C94B2040C942A0502FDFFC80002FCFF28
:1000F000C80002FBFFC80002FDFFC80002FCFFC8E9
:100100000002FBFFC80002FDFFC80002FCFFC800A0
:1001100002FBFFC80002FDFFC80002FCFFC800028E
:10012000FBFFC80002FDFFC80002FCFFC80002FB85
:10013000FFC80002FDFFC80002FCFFC80002FBFF71
:10014000C80002FDFFC80002FCFFC80002FBFFC898
:100150000002FDFFC80002FCFFC80002FBFFC80050
:1001600002FDFF900102FCFF900102FBFF900102E3
:10017000FDFFF40102FCFF260202FBFF580202FD14
:10018000FF200302FCFF840302FBFFE803000000E2
:10019000E803000000000002FEFF500002FDFF50D7
:1001A0000003FCFFAA000000001E0003FAFFAA00E3
:1001B0000000001E0003FAFFAA000000001E00025B
:1001C000FEFF500002FDFF500003FCFFAA000000EC
:1001D000001E0003FAFFAA000000001E0003FAFF41
:1001E000AA000000001E0002FEFF500002FDFF50AA
:1001F0000003FCFFAA000000001E0003FAFFAA0093
:100200000000001E0003FAFF2C0103FCFF82000324
:10021000FEFF8200000000500002FFFF500002FEBF
:10022000FF500003FDFFAA00000000140003FBFFC5
:10023000AA00000000140003FBFFAA000000001E3B
:100240000002FFFF500002FEFF500003FDFFAA0066
:10025000000000140003FBFFAA00000000140003CC
:10026000FBFFAA00000000140002FFFF500002FE86
:10027000FF500003FDFFAA000000001E0003FBFF6B
:10028000AA000000001E0003FBFF2C0103FDFF82FB
:100290000003FFFF8200000000500000000000008B
:1002A0000200006400020A00640002000064000210
:1002B0000A0064000200006400040000C800010A93
:1002C00000320001F6FF3200010A00320001F6FFA1
:1002D00032000200006400020A00640002000064B0
:1002E00000020A0064000200006400040000C8006C
:1002F000010A00320001F6FF3200010A003200015B
:10030000F6FF32000200006400020A0064000200EE
:10031000006400020A00640002000064000400009F
:10032000C800010A00320001F6FF3200010A003263
:100330000001F6FF32000200006400020A006400BF
:100340000200006400020A0064000200006400046D
:100350000000C800010A00320001F6FF3200010A65
:1003600000320001F6FF32000200006400020A00C1
:1003700064000200006400020A00640002000064DD
:1003800000040000C800010A00320001F6FF32003C
:10039000010A00320001F6FF320002FEFF64000293
:1003A0000800640002FEFF6400020800640002FE10
:1003B000FF6400040000C800010C00320001F8FFD7
:1003C0003200010C00320001F8FF320002FDFF6430
:1003D00000020700640002FDFF64000207006400E1
:1003E00002FDFF6400040000C800010D003200019E
:1003F000F9FF3200010D00320001F9FF3200000068
:10040000000000300C03DF31FA2B78D5D86C294579
:10041000A1026969918D6571B843DEF2F6786E1DAF
:10042000BF344ECB382EFD3259750732E231778416
:1004300033E1EDC56E5236279615198D8D88AB4D7B
:10044000BCF918F5271627818C2FB46E602BF29417
:100450000CE0597B338FA3C9A4BD573245027F02FC
:10046000FB98F723AE1EA53A4D59A9AE849B429145
:100470007C9B0CB02BB07ACF6DD102B2D381B4CEBD
:1004800019ACF2C7CB970218F0ABC774470906C482
:10049000A51374D0C3EEA030BFA2E2922497613DB1
:1004A0004453050FEA0728DAB3EF4FFAF955BE9F18
:1004B00068336F2B21105CE0B23F73D6D7D4141B86
:1004C000271A2A122153ECD5423CCF3C918EDBFAFD
:1004D000C24B26E35B82C40EC137E5980BFAB433F6
:1004E00014DE453631320B746EDBB1006A8CFA2CA7
:1004F000D7210F33A3D342650A27FE1621B249350F
:10050000918E6BC3C077382E52E92FBC7629E84D07
:100510004BF781EFCBC354D5EB53EC0D0635439825
:10052000C3AF5B842694B3787DE235F30C1D41574D
:1005300015C346E0879BB672EEA37FF5D8C28D9CAB
:1005400072E920987DD311FBB546EFC1643119796A
:10055000F45F5A7BFA11EEE9B46EDE8C316C29A39C
:1005600055493BD31C4DCED293BE94F7EFAD71E409
:100570000DCC6008DD4EF192BCD01FED3C4890924E
:1005800091CC65AE193481ADF215A5E2C317C6D082
:10059000E327D8C175CA53329B721FD8BBB06A4DCE
:1005A0007DD0FB97047D45F793EAD95601A027E457
:1005B000C700A53DCBF96F666C8F3F2740A974BE7D
:1005C0007A70557FEE9A76818550D787F1FF6BB9A7
:1005D000FF11F7CA0B673177F7709F371A14F6943B
:1005E000854B1373E68AF46CDBCBF3CCCB5F86CA06
:1005F000717D957CE4C6F4DC36931350A70AE52D93
:1006000055F9A03C8394A95F609C2B2BFCB2F66D3E
:10061000308BE91451DEF0887104D8190EBE46649F
:10062000B7E6A13B7B4A9ADBE7C607E378FD51A812
:10063000883BBDDA19AE628AB33AA4C2F9EB26B0A0
:10064000D2C8EC4D138629FA4D30DEC62E2F6FB678
:100650006A2D9083DBF20E8F2DB351279E78D871CF
:1006600040C4BE544BE84E98182D5F465DCEFDC782
:10067000FB8E4BD7815A66AF0EB7D6AC2FAE1D702E
:1006800072DCC4BDC41356DD40B6249D8421658050
:10069000B0B157310BBDE01975B6C6A564E415D7E6
:1006A000C1DA9585EDEC632EA287CC26A932A65936
:1006B000E3FD8AEFBB6B093021CFD586B4EB5D75C6
:1006C000C5F3FBB3DF5EE281E6AFA78FE14EE8C57D
:1006D0004C73B407DFBE38018E0D8742F8E5B8BE13
:1006E000D8B472B7125439F904E088E62F71AB7BA5
:1006F000E56083C41EBBC5ACC94DEFC233A7800CF7
:100700005BF3C36E48FC674CDDF0320D61DD88475A
:100710003E0B0B5CC7D109901EF852529FD25EFB74
:10072000C622690E1FD15AFDC28C0A236A926AA999
:100730009E760565470EF5660647B9A61A17A2E02C
:10074000390CEE59DD49569FD660C341F32EEA912C
:10075000A4F0F7ECFEEC5305340CAC4F244E2F5DA7
:100760005A1EB738670DD83E6D9C7F61CA69F26F1B
:1007700059E95C58D6B05E0BBC0A5AE0598A3EB4BF
:10078000A8F5EC1003C54E7161CED22C37C49C91F4
:10079000AEF8EA85A848906552EB46AC7584601EB9
:1007A0007A4D2F7D137DEE744CC0A183853D1534A9
:1007B00036FFBADF474B449A368A47AC0FA7CA893F
:1007C000F5F9070877F57DC3B61F473C5C5C71936C
:1007D0005C2B72A376B73EAC418558512D23DB22AA
:1007E0001CE22B93D8A8578FC79ECB24FB3CB7574E
:1007F000682AFBDEE1398B23BFE474EC074F0F243A
:10080000323AB87F8285888C8F9295989B9EA1A45E
:10081000A7AAADB0B3B6B9BBBEC1C3C6C9CBCED013
:10082000D3D5D7D9DCDEE0E2E4E6E8E9EBEDEEF0A3
:10083000F1F2F4F5F6F7F8F9FAFBFCFCFDFDFEFE2B
:10084000FEFEFEFEFEFEFEFEFDFDFCFCFBFAFAF9DE
:10085000F8F7F6F4F3F2F0EFEDECEAE8E7E5E3E1C0
:10086000DFDDDBD8D6D4D1CFCCCAC7C5C2BFBDBAB5
:10087000B7B4B1AFACA9A6A3A09D9A9693908D8A68
:100880008784817D7A7774716E6B6864615E5B5872
:1008900055524F4D4A4744413F3C393734322F2D52
:1008A0002A282623211F1D1B1917161412110F0E9B
:1008B0000C0B0A08070605040403020201010000EC
:1008C0000000000000000000010102020304050610
:1008D0000708090A0C0D0E1011131516181A1C1E04
:1008E00020222527292B2E303335383B3D404345E8
:1008F000484B4E5154575A5D606366696C6F72760F
:10090000797C7F0011241FBECFEFD1E2DEBFCDBFC7
:1009100000E00CBF84B78093460714BE0FB6F8946E
:10092000A8958091600088618093600010926000BB
:100930000FBE16E0A0E0B2E0EEEFF9E100E00BBF81
:1009400002C007900D92A63BB107D9F727E0A6EBAE
:10095000B6E001C01D92A634B207E1F70E94DC099F
:100960000C94FD0C0C940000CF93C62F0E944409F8
:100970008FEF80BBC1BBEBE0F1E08081857F80839E
:1009800085E08A95F1F7000080818A608083CF91AD
:1009900008950E94440910BA11BAEBE0F1E0808199
:1009A000837F808385E08A95F1F700008FB1908185
:1009B0009C609083089563E883E00E94B40463E040
:1009C00080E00E94B40460E081E00E94B40463E02F
:1009D00083E00E94B40480E092E090934307809308
:1009E00042078BEB92E00C94320ACF93DF93CDB7A2
:1009F000DEB7FE01369681919191BF010E945E0A99
:100A00008AE090E00E942C0A90E080E0DF91CF9194
:100A10000895CF92DF92EF92FF92CF93C82F80E498
:100A2000C82E82E4D82E8FE0E82EF12C85E00E94BB
:100A3000C90485FD06C081E0C81AD108E108F108A3
:100A4000A9F76C2F80E0CF91FF90EF90DF90CF90CF
:100A50000C94B404CF93C82F8A3019F48DE00E940F
:100A600009058C2F0E94090590E080E0CF91089540
:100A7000CF9385E00E94C90480FF0FC080E00E94F0
:100A8000C904C82F0E94B806CD3019F48AE00E942C
:100A900009058C2FCF910C940905CF910895CF9320
:100AA000C62F0E9444098FEF80BBC1BBEBE0F1E091
:100AB00080818D7E808385E08A95F1F700008081BA
:100AC00080618083808182608083CF9108950E94BD
:100AD000440910BA11BAEBE0F1E080818B7E80838B
:100AE00085E08A95F1F700008FB190819461908341
:100AF00008950F931F93CF93DF9380910F0283305C
:100B000009F4B3C0A8F4813009F444C0CFE78230BF
:100B100009F476C0C0E060E08C2F81700E944F0520
:100B2000CF5FCF3FC1F7DF91CF911F910F91089514
:100B3000843009F4C8C01FE7CFEFD0E00FEF853055
:100B400049F76091BC068FEF860F8E3F28F08091A9
:100B50000E02819580930E0280E00E944F05609105
:100B6000BC0681E00E944F054091B6065091B70641
:100B700057FDDFC08091BA069091BB06019684179D
:100B800095070CF0CAC09093BB068093BA0611502B
:100B9000C1F6C9CFCFE7E091BC06F0E0ED5FF74FBB
:100BA000649181E00E944F05E091BC06F0E0ED5FAA
:100BB000F74F649180E00E944F052091B606309176
:100BC000B70637FD19C08091BA069091BB06019611
:100BD000821793073CF49093BB068093BA06C150EA
:100BE000D1F6A1CF1092BB061092BA068091BC0636
:100BF0008F5F8093BC06F3CF8091BC06821BF9CF38
:100C00008091BC0687FF1DC06FEF80E00E944F05FA
:100C10006FEF81E00E944F052091B6063091B70634
:100C200037FD1FC08091BA069091BB0601968217CE
:100C300093076CF49093BB068093BA06C15001F7FA
:100C400072CF60E080E00E944F0560E0E2CF10923A
:100C5000BB061092BA068091BC068F5F8093BC06DB
:100C6000EDCF8091BC06821BF9CFCFE76091BC0627
:100C700080E00E944F056091BC0681E00E944F0514
:100C80002091B6063091B70637FD19C08091BA069B
:100C90009091BB060196821793073CF49093BB0694
:100CA0008093BA06C15011F73ECF1092BB06109246
:100CB000BA068091BC068F5F8093BC06F3CF80910B
:100CC000BC06821BF9CFCFE7E091B806F091B906D8
:100CD000ED5FFB4F649181E00E944F05E091B80603
:100CE000F091B906ED5FFB4F649180E00E944F05E3
:100CF0008091B8069091B9060196811524E092077B
:100D000038F49093B9068093B806C150E9F60BCF3A
:100D10001092B9061092B806F8CF1092BB06109246
:100D2000BA068091BC0690910E02890F8093BC0692
:100D30002ECF20910E022403B001259F700D1124A7
:100D40008091BC06FE01E81BF109E617F7071CF4C9
:100D50000093BC061CCF249F202D11242093BC0699
:100D600016CF80E00E94670580FF0C9479050895F6
:100D70009091BD06E92FF0E0E553F94F8F3729F444
:100D800091509093BD06108208959F5F9093BD0689
:100D900080830895FF920F931F93CF93DF93F62ED6
:100DA000C82FD0E08E01000F111FF801E758FD4F4A
:100DB00081818F9380818F930E94F504C15DD84F0C
:100DC0000F900F908881882311F0F11012C081E0FC
:100DD000888370E060E08AE00E942A05F801EB5900
:100DE000FD4F81818F9380818F930E94F5040F9036
:100DF0000F90DF91CF911F910F91FF900895CF93A6
:100E0000DF93C82FD0E0E091100284E0E89FF0016A
:100E10001124E35CFD4FEC0FFD1F808181110DC09B
:100E20008091AA028F938091A9028F930E94F5046A
:100E30000F900F90DF91CF910895FE01EE0FFF1FED
:100E4000E157FD4F81818F9380818F9381EC92E0F8
:100E50009F938F930E94F504E091100284E0E89F35
:100E6000F0011124E35CFD4FEC0FFD1F80818093A6
:100E7000100261E00E94CA06E0911002F0E0EE0F5D
:100E8000FF1FEF5EFD4F808191819093BF0680939D
:100E9000BE060F900F900F900F90CCCFEF92FF9265
:100EA0000F931F93CF93DF9309E317E0F80181912C
:100EB00081110DC087E0E034F807C9F784EE92E0B5
:100EC0009F938F930E94F5040F900F9028C08AED96
:100ED00092E09F938F930E94F5040F900F90D0E0C3
:100EE000C0E083EDE82E82E0F82EF80181918F01B9
:100EF000882389F0FE01EE0FFF1FE15DFD4F818128
:100F00008F9380818F93FF92EF920E94F5040F9050
:100F10000F900F900F902196C730D10531F7DF91D8
:100F2000CF911F910F91FF90EF900895E0911002E3
:100F3000F0E0EB5DFD4FE081E7FF0BC08091AE027A
:100F40008F938091AD028F930E94F5040F900F90C4
:100F50000895EE0FFF0BE15DFD4F81818F9380813E
:100F60008F938CEF92E09F938F930E94F5040F90E4
:100F70000F900F900F900895E0911002F0E0EB5D5C
:100F8000FD4FE081E7FF0BC08091AE028F9380910F
:100F9000AD028F930E94F5040F900F900895EE0F0D
:100FA000FF0BE15DFD4F81818F9380818F938BE0FB
:100FB00093E09F938F930E94F504E0911002F0E07C
:100FC000EB5DFD4FA0810A2E000CBB0BA75CB84F58
:100FD00081E08C938FEF80830F900F900F900F9094
:100FE0000895E82FF0E0E75CF84F9081911106C07A
:100FF0008091A6028F938091A5020FC08330C1F724
:10100000909110029230A1F710923C078093450214
:101010008091B6028F938091B5028F930E94F50460
:101020000F900F900895EF92FF920F931F93CF931D
:10103000DF93182F092F8FE2E82E82E0F82ED0E000
:10104000C0E0F701819191917F01FC0101900020A6
:10105000E9F73197AF01481B590B612F702F0E94A0
:10106000140A892B49F48C2FDF91CF911F910F9196
:10107000FF90EF900C94F1072196C730D10509F746
:101080008091A6028F938091A5028F930E94F50410
:101090000F900F90DF91CF911F910F91FF90EF90E4
:1010A00008950F931F93CF93DF93C82F70E060E0F4
:1010B0008AE00E942A05C73009F446C0A8F5C53069
:1010C000D1F1C63009F446C08FEF8C0F8430C8F1DF
:1010D0008BE193E09F938F930E94F504CDE8D2E0DB
:1010E0000F900F9003ED12E08881998122969F93D3
:1010F0008F931F930F930E94F5040F900F900F9002
:101100000F9082E0C13AD80779F78091A8028F93B7
:101110008091A7028F930E94F5040F900F90DF91AA
:10112000CF911F910F910895C83089F0C93081F691
:101130000E94BC07EACF60E0809110020E94CA06BC
:10114000E4CF0E94FF06E1CF0E944E07DECF0E944F
:101150009607DBCFE0919902F0919A02DF010D90A2
:101160000020E9F7CD018E1B9F0B8553994F0E94FC
:101170001308CBCF0F931F93CF93DF93E091BD065E
:10118000E436B0F01092BD06EBECF6E084E6DF0149
:101190001D928A95E9F784E293E09F938F930E94D2
:1011A000F5040F900F90DF91CF911F910F9108954B
:1011B000F0E0E653F94F80818A3011F08D3099F7D5
:1011C0000DE812E0D0E0C0E0F801819191918F012B
:1011D000FC0101900020E9F73197AF01481B590B42
:1011E0006BEC76E00E94140A892B69F48C2F0E9424
:1011F00051081092BD06EBECF6E084E6DF011D928B
:101200008A95E9F7D0CF2196CA30D105E9F68091C9
:10121000A4028F938091A3028F930E94F5040F90F4
:101220000F90E7CF82E884BD84E085BD80E487BD70
:1012300082E080936E0008951F920F920FB60F9276
:1012400011240BB60F922F933F934F935F936F939D
:101250007F938F939F93AF93BF93EF93FF930E94DE
:101260006909FF91EF91BF91AF919F918F917F910C
:101270006F915F914F913F912F910F900BBE0F9007
:101280000FBE0F901F9018958093080108958FEF5F
:1012900080BB8093070180930A011092080111BA64
:1012A000EBE0F1E0108280818F6180838FE891E034
:1012B0000197F1F700C0000080818E7F8083089540
:1012C0000E94B1060E9438050E94BA0890E080E0B2
:1012D00008956091BE067091BF066115710529F4ED
:1012E0001092CA061092C90608958091C90690917D
:1012F000CA0601969093CA068093C9062091C20639
:101300003091C3064091C7065091C80684179507CF
:1013100020F46217730721F408956217730761F0D0
:101320001092C1061092C0061092CA061092C90609
:101330007093C3066093C2062091C0063091C10627
:1013400045E0429FC001439F900D1124680F791F13
:1013500045E050E084EC96E00E940B0A8091C706BD
:101360009091C806892B71F41092C1061092C006A4
:101370006091BE067091BF0645E050E084EC96E0B7
:101380000E940B0A8091C40680930F028091C506CB
:101390009091C6069093B7068093B6061092CA063F
:1013A0001092C9068091C0069091C1060196909353
:1013B000C1068093C0060895F8940E9447090E94D0
:1013C000DB040E94120988EE90E09093BF068093A0
:1013D000BE06EFE2F7E08AE0DF011D928A95E9F7A9
:1013E000E9E3F7E087E0DF011D928A95E9F760E025
:1013F000809110020E94CA06789488E19EE00FB6A0
:10140000F894A895809360000FBE90936000A89513
:101410000E946009FCCFFB01DC0102C005900D9227
:1014200041505040D8F70895FB01DC014150504035
:1014300088F08D9181341CF08B350CF4805E6191C5
:1014400061341CF06B350CF4605E861B611171F326
:10145000990B0895881BFCCF609142077091430758
:101460000C946F0C0F931F93CF93DF93E09142077F
:10147000F0914307238110E000E021FD0EC00FEF43
:101480001FEFC801DF91CF911F910F91089519951A
:10149000892B11F00FEF1FEFCE01EC0189916091C4
:1014A000420770914307DB011896ED91FC91811181
:1014B000EECF8AE01995892B21F3E1CFAB01BC0176
:1014C00080914207909143070C94660A2F923F92B5
:1014D0004F925F926F927F928F929F92AF92BF9244
:1014E000CF92DF92EF92FF920F931F93CF93DF93F0
:1014F00000D000D000D00F920F92CDB7DEB77C01A4
:101500003B018A01FC0117821682838181FFCEC1D3
:101510009AE0292ECE0101965C01F7019381F30137
:1015200093FD859193FF81913F01882309F446C182
:10153000853239F493FD859193FF81913F01853286
:1015400029F4B70190E00E946F0CE7CF912C412C59
:10155000512CFFE1F51538F08B3209F188F4803217
:1015600001F1833221F157FC3AC020ED280F2A30D7
:1015700040F556FE1FC0929C200D1124922E06C0ED
:101580008D3291F0803379F7689450F8F30193FD30
:10159000859193FF81913F018111DBCF20C0689439
:1015A00051F8689452F8F2CF689453F8EFCF6894EA
:1015B00054F8ECCF429C200D1124422E689455F82B
:1015C000E5CF8E3229F456FCF9C0689456F8DECF88
:1015D0008C3619F4689457F8D9CF8836B9F2982F19
:1015E0009F7D95549330C0F08336A1F18337C1F1CC
:1015F000833509F05BC0F801C190D1908F01692D4E
:1016000070E056FC02C06FEF7FEFC6010E94590CDC
:101610004C01689457F80AC00C5F1F4F2FE32983D1
:1016200088248394912C6501E89457F853FC04C0F6
:101630004814190409F018F5342C8114910431F57B
:10164000332009F46ACFB70180E290E00E946F0C6A
:101650003A94F6CFF801808189830E5F1F4FE0CF67
:10166000F801C190D1908F01692D70E056FC02C045
:101670006FEF7FEFC6010E94640C4C01D5CFB7011C
:1016800080E290E00E946F0C4A94D2CFF60157FCA2
:10169000859157FE81916F01B70190E00E946F0C18
:1016A00031103A94F1E08F1A9108C7CF843619F0BF
:1016B000893609F074C0F80157FE6AC061917191D2
:1016C000819191918F01252D2F76D22E97FF09C000
:1016D00090958095709561957F4F8F4F9F4F68943F
:1016E000D7F82AE030E0A5010E949F0CC82ECA1846
:1016F0008C2C5D2CD6FE0CC0E89450F8C91440F434
:10170000D4FE05C0D2FC03C0FD2DFE7E5F2E892CC9
:1017100054FEA4C0FE01EC0DF11D8081803309F060
:1017200096C0252D297E522E852D8870382E53FC8B
:10173000A4C050FE9EC09C2C841418F44C0C942C15
:10174000981854FEA0C0B70180E390E00E946F0C8F
:1017500052FE09C088E790E051FE02C088E590E0A3
:10176000B7010E946F0CC91408F499C0CA94D12C17
:101770009FEFC91AD90ACA0CDB1CF60182916F01CE
:10178000B70190E00E946F0CAC14BD04B1F758CFC4
:1017900061917191072E000C880B990B93CFD52C7A
:1017A000E894D4F82AE030E08537E1F1952D997F6F
:1017B000D92E8F36A9F1F0F4883551F1F7018681E1
:1017C00097812B960FB6F894DEBF0FBECDBFDF9189
:1017D000CF911F910F91FF90EF90DF90CF90BF902E
:1017E000AF909F908F907F906F905F904F903F90C1
:1017F0002F900895803749F0883701F7D4FE02C052
:101800006894D2F820E130E00DC06894D4F8F6CFA7
:1018100054FE03C0E92FE660DE2E20E132E002C074
:1018200028E030E0F801D7FE0DC0619171918191FF
:1018300091918F01A5010E949F0CC82ECA18E894AF
:10184000D7F856CF6191719190E080E0F2CF52FCD1
:1018500002C0839469CF8394839466CF852D867864
:1018600009F462CFF6CFB70180E290E00E946F0CDE
:1018700083948414C0F3312C64CF342C381884142E
:1018800008F45FCFF8CF852D867809F46CCF8BE212
:1018900051FE80E257FC8DE2B70190E062CFB701C4
:1018A00080E390E00E946F0C9A945DCF8FEF9FEFE2
:1018B00088CFFC010590615070400110D8F78095E9
:1018C00090958E0F9F1F0895FC016150704001900C
:1018D0000110D8F7809590958E0F9F1F08950F9354
:1018E0001F93CF93DF93182F092FEB018B8181FD7D
:1018F00009C01FEF0FEF812F902FDF91CF911F9124
:101900000F91089582FF14C02E813F818C819D81AB
:10191000281739073CF4E881F981CF0101969983B2
:10192000888310838E819F8101969F838E83E3CF6E
:10193000E885F985812F1995892BA1F3DACFFA0172
:10194000AA27283051F1203181F1E8946F936E7FFE
:101950006E5F7F4F8F4F9F4FAF4FB1E03ED0B4E0EF
:101960003CD0670F781F891F9A1FA11D680F791F30
:101970008A1F911DA11D6A0F711D811D911DA11D41
:1019800020D009F468943F912AE0269F1124301951
:10199000305D3193DEF6CF010895462F4770405DEC
:1019A0004193B3E00FD0C9F7F6CF462F4F70405D9B
:1019B0004A3318F0495D31FD4052419302D0A9F7F6
:1019C000EACFB4E0A6959795879577956795BA95F0
:1019D000C9F700976105710508959B01AC010A2EB6
:1019E00006945795479537952795BA95C9F7620F8D
:0E19F000731F841F951FA01D0895F894FFCF4C
:1019FE0000000002000000002A05000000000101A6
:101A0E0001E8009701A002000000000000000000A5
:101A1E000000000000FF0603FFFFFFFFFFFFFF3582
:101A2E000341034E0352035A03600369030000008F
:101A3E00000200000000010000000004020000008F
:101A4E000000000000000000000000000000000088
:101A5E000000000000700313049B04260530053BB4
:101A6E000545055105570560056E05760582052667
:101A7E000590053B0545055105570560059B05A0DD
:101A8E0005A605AC05B105B605BF05C305CD05D444
:101A9E0005D905DF05F00504061E06350646065E69
:101AAE00066606720688069706A606494E49540D26
:101ABE00004D6F76696E6720746F77617264732064
:101ACE0025730020202020257300596F7520686132
:101ADE0076653A00596F757220696E76656E746F11
:101AEE00727920697320656D70747900596F752055
:101AFE00666F756E64206120257300596F752074B2
:101B0E006F6F6B2074686520257300596F752063A5
:101B1E00616E3A000A546F6F206D75636820696EAE
:101B2E007075742100464C4F505059204449534B08
:101B3E0000534352455720445249564552004B4597
:101B4E0059005341555341474500464C45534800B3
:101B5E004B4559424F41524400504953544F4C004B
:101B6E00596F7520737461726520696E746F206190
:101B7E0020766F6964206F66206E6F7468696E6779
:101B8E006E6573732E20596F7520736565206E6FA9
:101B9E006F6E652C20796F752068656172206E6F8F
:101BAE006F6E652C796F75206665656C20736F6D31
:101BBE00656F6E652E0A596F75206C6F6F6B2061A5
:101BCE00726F756E642C20616E6420736565206E75
:101BDE006F7468696E672C2079657420796F752033
:101BEE00617265206E6F206C657373207363617212
:101BFE0065642E20596F75206861766520776F6E4B
:101C0E002E2E00596F7520617265206F6E207468DC
:101C1E0065206465616420656E64206F66206120B6
:101C2E006C6F6E656C7920726F61642E20596F75C2
:101C3E00206C6F6F6B20726967687420616E642010
:101C4E006C656674206F66796F752C206275740AE8
:101C5E00796F752063616E6E6F742072656D656D40
:101C6E006265722077687920796F752061726520C0
:101C7E00686572652E2E2E20596F75206172652053
:101C8E007465727269666965642E00596F75207489
:101C9E00726176656C20612062697420746F776161
:101CAE0072647320746865206D6F6F6E2C20796F6F
:101CBE0075207468696E6B20746861742773207464
:101CCE0068652077617920746F20676F2E20596FB9
:101CDE00752066696E642061200A626561722069F2
:101CEE006E20746865206D6964646C65206F662073
:101CFE0074686520726F616420736C656570696EBF
:101D0E0067207365656D696E676C7920696E2070EA
:101D1E00656163652E0046495245504C414345006E
:101D2E00572F5720535452454554004F4C4420488A
:101D3E004F555345004C4956494E4720524F4F4D33
:101D4E0000415454494300424153454D454E5400C1
:101D5E00434F4D505554455220524F4F4D004E4F0C
:101D6E005448494E47004C4F4E454C5920524F4116
:101D7E004400532F4E204449525420524F414400A8
:101D8E00452F57205374726565740068656C70003A
:101D9E006E6F72746800736F757468007765737414
:101DAE0000656173740064657363726962650075C2
:101DBE00736500696E76656E746F72790073656116
:101DCE007263680074616B65004552524F52004950
:101DDE006E76616C696420636F6D6D616E64210057
:101DEE00596F752063616E27742075736520746852
:101DFE0061742100576861742061726520796F7576
:101E0E0020676F696E6720746F20646F3F00596F93
:101E1E00752063616E277420676F2074686174206B
:101E2E007761792100594F55204D41592041435436
:101E3E00204E4F5721005468657265206973206EDD
:101E4E006F7468696E6720686572652E2E006974FE
:101E5E0020646965640069742073757276697665AD
:101E6E00640061206265617220626C6F636B732027
:101E7E00746865207761790069742072616E2061E3
:101E8E007761792E2E2E00697420776F6E2774205D
:101E9E00737461727400796F752063616E2774209C
:061EAE007479706500006C
:00000001FF
